:100000000C947B050C94C3050C94C3050C94C30598
:100010000C94C3050C94C3050C94C3050C94C30540
:100020000C94C3050C94C3050C94C3050C94A60F43
:100030000C94C3050C94A11D0C94C3050C94C3052A
:100040000C94C3050C94C3050C94C3050C94FA1DC1
:100050000C94C3050C94C3050C94C3050C945A0866
:100060000C94C3050C94C3050C94C3050C94C305F0
:100070000C94C3050C0E330E2B0F330E2B0F7F0E7B
:10008000A20E2B0FF90E080FC913C9130114011486
:100090007C14B014A716A716C714A7165814581422
:1000A0006116A7167616941688000000000000005E
:1000B0000400050006000700080009000A000B0004
:1000C0000C000D000E000F001000110012001300B4
:1000D0001400150016001700180019001A001B0064
:1000E0001C001D001E001F00200021002200230014
:1000F0002400250026002700280029002A002B00C4
:100100002C002D002E002F003000310000003300A5
:100110003400000036003700380082003A003B000F
:100120003C003D003E003F004000410042004300D3
:100130004400450046000000000049004A004E000F
:100140004C004D004B004F00500051005200000089
:100150005400550056005700580059005A005B00E3
:100160005C005D005E005F00600061006200630093
:100170000000650085006700680069006A000000F3
:10018000000000000000000000000000000000006F
:10019000890087008A008B00E000E100E200E300B4
:1001A0000000E500E600E700291E1F20212223248D
:1001B0002526272D2E742A2B141A0815171C180C07
:1001C00012132F3028041607090A0B0D0E0F3334B3
:1001D000311D1B0619051110363738752C764E4B1C
:1001E000494C52504F514A4D56545F6061555C5DC9
:1001F0005E57595A5B6762666377444568696A80EF
:10020000707172738080658048463A3B3C3D3E3F4A
:1002100040414243808080807939007A7880807BB9
:100220007F7E8080807D8080706339385F6C6564FC
:100230003A20253032580A007573625F6C65643A63
:1002400020253032580A0073656E642025303258FC
:100250003A20253032580A0073656E642039443ADA
:1002600020253032580A007225303258200073653C
:100270006E642037303A20253032580A0073656E9C
:10028000642039433A20253032580A007225303430
:10029000582000732530325820006F6C6420747928
:1002A00070650A006E657720747970650A000A4BE4
:1002B0006579626F6172642073746172742E0A00D2
:1002C0000A55534220636F6E666967757265642EC6
:1002D0000A000A0A544D4B3A64373362656462354A
:1002E0002F4C5546410A0A003003500043003900A4
:1002F000380020006B006500790062006F0061002B
:1003000072006400200063006F006E0076006500DC
:10031000720074006500720000000E0374002E006D
:100320006D002E006B002E0000000403090409027A
:100330007400040100A0320904000001030101005F
:100340000921110100012240000705810308000A6C
:100350000904010001030102000921110100012229
:100360004D000705820308000A090402000103008A
:10037000000009211101000122360007058303084E
:10038000000A090403000203000000092111010012
:100390000122220007058403200001070504032031
:1003A00000011201100100000008EDFE019801019A
:1003B000010200010631FF0974A10109751500262B
:1003C000FF009520750881020976150026FF00952B
:1003D0002075089102C005010980A101850216015E
:1003E000002637001A81002AB70075109501810098
:1003F000C0050C0901A1018503160100269C021A03
:1004000001002A9C02751095018100C005010902B6
:10041000A1010901A10005091901290515002501FE
:10042000950575018102950175038101050109306A
:1004300009311581257F95027508810609381581D6
:10044000257F950175088106050C0A38021581255E
:100450007F950175088106C0C005010906A1010547
:100460000719E029E7150025019508750181029516
:100470000175088101050819012905950575019186
:10048000029501750391010507190029FF15002642
:10049000FF00950675088100C0636F6E73756D650A
:1004A000723A20253034580A0073797374656D3AB6
:1004B00020253034580A000A002530325820006BBD
:1004C0006579626F6172643A20004C45443A202598
:1004D0003032580A0025583A2530386225730A0010
:1004E0000A202030313233343536370A00290A00E9
:1004F0002575002F002575005D280025640020006B
:10050000256400200025640020002564007C00256F
:10051000303258006D6F7573656B6579205B62745E
:100520006E7C782079207620685D287265702F6156
:10053000636C293A205B006D6B5F776865656C5F63
:1005400074696D655F746F5F6D6178203D2025640F
:100550000A006D6B5F776865656C5F6D61785F73CE
:1005600070656564203D2025640A006D6B5F7469C9
:100570006D655F746F5F6D6178203D2025640A00B2
:100580006D6B5F6D61785F7370656564203D2025DC
:10059000640A006D6B5F696E74657276616C203DF4
:1005A0002025640A006D6B5F64656C6179203D20D5
:1005B00025640A006D6B5F776865656C5F74696DB3
:1005C000655F746F5F6D6178203D2025640A006D62
:1005D0006B5F776865656C5F6D61785F737065658B
:1005E00064203D2025640A006D6B5F74696D655F52
:1005F000746F5F6D6178203D2025640A006D6B5F2C
:100600006D61785F7370656564203D2025640A0024
:100610006D6B5F696E74657276616C203D20256438
:100620000A006D6B5F64656C6179203D2025640A6A
:10063000000A00257500363A20776865656C5F749E
:10064000696D655F746F5F6D61783A20000A0025FF
:100650007500353A20776865656C5F6D61785F730A
:10066000706565643A20000A00257500343A2074EC
:10067000696D655F746F5F6D61783A20000A0025CF
:100680007500333A206D61785F73706565643A2058
:10069000000A00257500323A20696E746572766131
:1006A0006C286D73293A20000A00257500313A2024
:1006B00064656C6179282A31306D73293A20000A0B
:1006C000092D2056616C756573202D0A004D3E0082
:1006D0004D25643E20003F007365742064656661AB
:1006E000756C740A00433E2000776865726520646B
:1006F000656C74613A20637572736F723D25642C6A
:1007000020776865656C3D25640A536565206874CB
:1007100074703A2F2F656E2E77696B697065646906
:10072000612E6F72672F77696B692F4D6F757365D7
:100730005F6B6579730A000A092D204D6F7573652B
:100740006B6579202D0A4553432F713A09717569FC
:10075000740A313A0964656C6179282A31306D7305
:10076000290A323A09696E74657276616C286D7374
:10077000290A333A096D61785F73706565640A34DC
:100780003A0974696D655F746F5F6D61780A353A17
:1007900009776865656C5F6D61785F737065656426
:1007A0000A363A09776865656C5F74696D655F74D0
:1007B0006F5F6D61780A0A703A097072696E742011
:1007C00076616C7565730A643A09736574206465B3
:1007D0006661756C74730A75703A092B310A646F1F
:1007E000776E3A092D310A706775703A092B3130EE
:1007F0000A7067646F776E3A092D31300A0A737098
:10080000656564203D2064656C7461202A206D61FB
:10081000785F7370656564202A2028726570656151
:1008200074202F2074696D655F746F5F6D61782926
:100830000A003F004D3E2000433E20004C25640A44
:10084000000A092D20436F6E736F6C65202D0A45D9
:1008500053432F713A09717569740A6D3A096D6FC6
:100860007573656B65790A000A092D204D6167690A
:1008700063202D0A643A0964656275670A783A094B
:100880006465627567206D61747269780A6B3A09F4
:100890006465627567206B6579626F6172640A6D69
:1008A0003A096465627567206D6F7573650A763AFB
:1008B0000976657273696F6E0A733A0973746174AD
:1008C00075730A633A09636F6E736F6C65206D6FA1
:1008D00064650A302D343A096C61796572302D34C3
:1008E000284631302D4634290A506175733A096221
:1008F0006F6F746C6F616465720A003F0074696D9C
:1009000065725F72656164333228293A202530347C
:100910006C580A006B6579626F6172645F69646C20
:10092000653A2025580A006B6579626F6172645FD1
:1009300070726F746F636F6C3A2025580A00686F8D
:1009400073745F6B6579626F6172645F6C65647309
:1009500028293A2025580A000A092D205374617469
:100960007573202D0A004743433A20352E342E302C
:10097000204156522D4C4942433A20322E302E30DF
:10098000204156525F415243483A206176723335D6
:100990000A004F5054494F4E533A204C554641207F
:1009A0004D4F5553454B45592045585452414B45A1
:1009B0005920434F4E534F4C4520434F4D4D414ED0
:1009C0004420343039360A004255494C443A2064B8
:1009D00037336265646235202831353A35333A3031
:1009E00033204A616E2031372032303231290A00FB
:1009F0005649443A2030784645454428742E6D2E99
:100A00006B2E29205049443A20307839383031282B
:100A100050433938206B6579626F61726420636F6F
:100A20006E76657274657229205645523A20307888
:100A3000303130310A00444553433A20636F6E76BB
:100A4000657274732050433938206B6579626F6129
:100A500072642070726F746F636F6C20696E746F54
:100A6000205553420A000A092D2056657273696F9A
:100A70006E202D0A000A6D6F7573653A206F6666E9
:100A80000A000A6D6F7573653A206F6E0A000A6B73
:100A90006579626F6172643A206F66660A000A6B5C
:100AA0006579626F6172643A206F6E0A000A6D6147
:100AB000747269783A206F66660A000A6D61747212
:100AC00069783A206F6E0A000A64656275673A2099
:100AD0006F6E0A000A64656275673A206F66660A7F
:100AE000000A0A626F6F746C6F616465722E2E2E3D
:100AF0002000433E200011241FBECFEFD4E0DEBF14
:100B0000CDBF04B603FE28C080915A0490915B04C7
:100B1000A0915C04B0915D048730904BA740B04B2E
:100B2000D9F410925A0410925B0410925C04109253
:100B30005D0414BE0FB6F894A8958091600088619A
:100B400080936000109260000FBE10920108109216
:100B50000008E0E0F8E3099511E0A0E0B1E0E2E28E
:100B6000FDE402C005900D92A833B107D9F724E047
:100B7000A8E3B1E001C01D92AA35B207E1F70E94D7
:100B80002B0B0C948F260C940000FF93EF93E091B5
:100B90003801F0913901309709F00995EF91FF91F3
:100BA0000895FC018591803011F0EFDFFBCF0895AF
:100BB000FF27E0E230E247FF0CC0419597FF09C0F4
:100BC000EDE26095709580959095611D711D811D78
:100BD000911D27FF02C0219530E350E2AA27660F3E
:100BE000771F881F991FAA1FA41710F0A41B6395D5
:100BF0005A95A9F7AA3008F0A95FA05DAF93F395C5
:100C0000611571058105910541F7ED3211F4EF93FE
:100C1000F395F21718F43F93F395FBCF8F91B5DF5F
:100C2000FA95E1F70895E991F9918591803021F0E5
:100C3000853219F0AADFF9CF089520E0E8945591A4
:100C40005532C1F3503311F4689455915A3348F436
:100C5000505390F3220F022E220F220F200D250F4A
:100C6000F4CF0EF4219589919991533619F35337A6
:100C700029F1533559F1BC0188279927E8945C364E
:100C800021F48991999168945591543639F446EF3D
:100C90007EF077FF0DC08FEF9FEF0AC055374AE017
:100CA00039F0583540E121F0523642E009F008951C
:100CB000FF93EF937DDFEF91FF91B7CFFF93EF931A
:100CC000FC0181918030B9F360DFFBCFFF93EF939C
:100CD00068DFF1CFDF93CF93CDB7DEB72596A3DFE3
:100CE000CF91DF910895CF93C82F1F928F9383E9FF
:100CF00092E09F938F930E946A065C9A8FE99FE02F
:100D00000197F1F700C000008C2F0E9453088FE973
:100D10009FE00197F1F700C000005C980F900F90E2
:100D20000F900F90CF9108951F93CF93DF931FEFF4
:100D30000E943F08EC011150CF3F9FEFD90741F4CB
:100D40008FE99FE00197F1F700C000001111F0CF8B
:100D50005C9A85ED8A95F1F700005C98DF93CF935C
:100D60008CE892E09F938F930E946A060F900F90F9
:100D70000F900F90CE01DF91CF911F910895EF92C8
:100D8000FF920F931F93CF93DF93539A549A519AE4
:100D90005B9A5C9A599A0E9429085C9A5B9820E5B4
:100DA0002A95F1F75B9A8FEF90E722E0815090400F
:100DB0002040E1F700C000008FE90E9473060E9406
:100DC00094068A3F910569F40E949406803A910541
:100DD00041F40E9494068038910519F484EA92E067
:100DE00002C08AE992E09F938F930E946A060F9057
:100DF0000F900DE712E08EE6E82E82E0F82E8CE9E7
:100E00000E9473060E949406EC01CF3F8FEFD80733
:100E100029F4EBE3F1E08BE491E02DC080913C04F8
:100E200080FF0AC0DF93CF931F930F930E946A063F
:100E30000F900F900F900F90CA3FD10551F780E7A8
:100E40000E9473060E949406EC01CF3F8FEFD807F3
:100E5000B1F280913C0480FF0AC0DF93CF93FF92F0
:100E6000EF920E946A060F900F900F900F90CA3F6A
:100E7000D10529F6CECF11928E179F07E1F75C9826
:100E8000DF91CF911F910F91FF90EF900895EF9216
:100E9000FF920F931F93CF93DF930E943F08F82E8A
:100EA000082F192F0F3F8FEF180709F04EC08091C0
:100EB0003A01882309F48FC008E512E097E4E92E8F
:100EC00092E0F92E8DE90E9473060E949406EC01CF
:100ED000CF3F8FEFD80721F410923A0180E07BC01A
:100EE00080913C0480FF0AC0DF93CF931F930F9340
:100EF0000E946A060F900F900F900F90CA3FD10585
:100F000059F780913A010E9473060E949406EC0101
:100F1000CF3F8FEFD807B1F280913C0480FF10C023
:100F2000DF93CF9380913A011F928F93FF92EF92BC
:100F30000E946A060F900F900F900F900F900F90E5
:100F4000CA3FD10509F0BECFC7CF9F93FF9287E676
:100F500092E09F938F930E946A060F900F900F90DC
:100F60000F90E80183E0D695C7958A95E1F76F2D3C
:100F700067708C2F8F70F7FE14C00E94D6118823E3
:100F800019F1CF70DD27C55CDE4F0770112781E0B6
:100F900090E001C0880F0A95EAF78095988189232F
:100FA00012C00E94D61181110FC0CF70DD27C55C21
:100FB000DE4F0770112781E090E001C0880F0A958D
:100FC000EAF79881892B88835C9A85ED8A95F1F7F9
:100FD00000005C988F2DDF91CF911F910F91FF90B2
:100FE000EF900895E82FF0E0E55CFE4F80810895D2
:100FF00080FD02C090E701C091E790933A0181FF24
:1010000005C090913A01946090933A0190913C040C
:1010100090FF0CC01F928F9388E392E09F938F9371
:101020000E946A060F900F900F900F9080913C04E1
:1010300080FF0EC080913A011F928F9388E292E068
:101040009F938F930E946A060F900F900F900F90BE
:10105000089583E38093CC001092CD00E9ECF0E09A
:10106000808180698083808188608083EAECF0E001
:1010700080818063808352985A9A78940895209151
:101080004B0180914C01821759F030E0F901E35B8C
:10109000FE4F80812F5F3F4F20934B0190E00895DA
:1010A0008FEF9FEF08959091C80095FFFCCF80933C
:1010B000CE0008951F920F920FB60F9211242F9316
:1010C0003F934F938F939F93EF93FF9380914C01A6
:1010D00090E09C012F5F3F4F40914B01421741F040
:1010E0003091CE00FC01E35BFE4F308320934C0136
:1010F000FF91EF919F918F914F913F912F910F9081
:101100000FBE0F901F901895809158030895CF93AC
:10111000DF9300D01F92CDB7DEB79C0180915104C0
:10112000843019F593E099833B832A839093E900F7
:101130008FEF9091E800815095FD06C095ED9A954E
:10114000F1F700008111F5CF8091E80085FF0DC017
:1011500040E050E063E070E0CE0101960E94DD0CBB
:101160008091E8008E778093E8000F900F900F90A9
:10117000DF91CF910895CF93DF9300D01F92CDB729
:10118000DEB720915104243031F522E029838058C4
:1011900091099B838A8383E08093E9008FEF90918C
:1011A000E800815095FD06C095ED9A95F1F7000095
:1011B0008111F5CF8091E80085FF0DC040E050E03F
:1011C00063E070E0CE0101960E94DD0C8091E800A2
:1011D0008E778093E8000F900F900F90DF91CF9162
:1011E0000895209151042430F1F422E02093E90085
:1011F0002FEF3091E800215035FD06C035ED3A95CE
:10120000F1F700002111F5CF2091E80025FF0BC078
:1012100040E050E065E070E00E94DD0C8091E80065
:101220008E778093E8000895CF93DF932091510447
:10123000243049F521E02093E90021E8215059F0BC
:101240003091E80035FD07C0EFE3F1E03197F1F7A9
:1012500000C00000F3CF2091E80025FF14C0EC018E
:1012600040E050E068E070E00E94DD0C8091E80012
:101270008E778093E80088E0FE01A0E5B3E001905E
:101280000D928A95E1F7DF91CF910895CF93C091A8
:101290004F02C1110BC00E94DF1D643C79408105E3
:1012A000910520F081E080934F02C1E08C2FCF9117
:1012B0000895FF920F931F93CF93DF93D82F0FB60C
:1012C00007FE83C080915104843081F08091030136
:1012D00090E001962091050130E082239323209134
:1012E000040130E08217930709F0C9C00E94460943
:1012F000811110C08091030190E0019620910501B9
:1013000030E0822393232091040130E08217930779
:1013100009F0B5C00E94D31D8C01C091E900CF70C7
:101320009091EC00892F817090FD80E8C82B84E0BB
:101330008093E90085E0F82E8091EB0085FD42C0A6
:101340008091EB0080FF3EC08091EE0087FF3AC0A5
:101350008091040190910301981709F457C090916E
:10136000E80095FF8AC0E0910101F0910201E80FC9
:10137000F11D20818F5F90910501892380930401E5
:101380002093F1008091E80085FDE2CF8091E80094
:1013900080FFDECF8091E8008E778093E800F092A6
:1013A0000001D6CF8091030190E0019620910501C4
:1013B00030E0822393232091040130E082179307C9
:1013C00009F448C0CF70C093E90040910301842F15
:1013D00090E001962091050130E082239323209133
:1013E000040130E08217930709F44CC0E091010139
:1013F000F0910201E40FF11DD083809103018F5F12
:10140000909105018923809303013CC08091E800FD
:1014100085FF33C0D093F10081E09091F2009923D1
:1014200091F09091E80090FF0EC09091E80095FF38
:1014300003C01092F100F9CF9091E8009E7790934D
:10144000E800F0920001882309F4ACCFCF70C0937C
:10145000E90018C080910001882309F4B3CF0E94ED
:10146000D31D9C018017910711F4890165CF9091DC
:101470000001915090930001F8CF80E0CECF4091D1
:101480000301B4CF80E0DF91CF911F910F91FF90C6
:10149000089580915004811104C00E94430F0C9460
:1014A000960F0895109250040895089542E061EC5B
:1014B00081E00E94560C42E061EC82E00E94560CF2
:1014C00042E061EC83E00E94560C42E261EC84E071
:1014D0000C94560C80915304833009F453C030F4BB
:1014E000813071F0823009F48CC008958A3009F49B
:1014F00078C08B3009F45EC0893009F09AC020C0F2
:1015000080915204813A09F094C08091E800877F6D
:101510008093E8008091560490915704892B21F420
:1015200068E080E593E003C060E080E090E070E078
:101530000E942A0D8091E8008B778093E80008953F
:1015400080915204813209F074C0809156049091C8
:101550005704892B09F06DC08091E800877F809344
:10156000E8008091E80082FD05C08091510481115E
:10157000F8CF5FC08091F100809358038091E8001C
:101580008B7753C080915204813A09F052C0809108
:10159000560490915704892B09F04BC08091E800C4
:1015A000877F8093E8008091E80080FFFCCF8091E6
:1015B000100136C0809152048132D9F580915604D1
:1015C00090915704892BA9F58091E800877F80933B
:1015D000E8000E948B0C80915404809310010C94BD
:1015E000791380915204813221F58091E800877F40
:1015F0008093E8000E948B0C8091550480935903DE
:10160000089580915204813AA1F48091E800877F87
:101610008093E8008091E80080FFFCCF809159031F
:101620008093F1008091E8008E778093E8000C941D
:101630008B0C08950E94641D80914F04882329F02B
:101640000E948D1D81110C94400C089508950C94F6
:10165000260B0C94260BCF9384B7877F84BF0FB6DD
:10166000F894A89580916000886180936000109242
:1016700060000FBE90E080E80FB6F89480936100A0
:10168000909361000FBE89E599E00E94371D86E0C6
:1016900091E00E946B1082ED92E00E94D1050E94C1
:1016A000290B0E942A110E94430F0E94960F7894E2
:1016B0000E942C1180915104843029F00E94501016
:1016C0000E94260BF7CF80EC92E00E94D1050E9489
:1016D000270B8EEA92E00E94D105C4E0809151046C
:1016E000853019F40E941A0BF9CF0E943011209115
:1016F000E4003091E50080914D0290914E02281750
:10170000390709F464C08091E4009091E50090935A
:101710004E0280934D020E944609882309F457C067
:1017200080915104843009F052C08091E9008F709B
:101730002091EC00922F917020FD90E8892BC093AE
:10174000E9009091EB0090FF3FC09091EE0097FF71
:101750003BC09091040120910301291709F12091C8
:10176000E80025FF1DC0E0910101F0910201E90FA1
:10177000F11D30819F5F2091050192239093040118
:101780003093F1009091E80095FDE3CF9091E8004F
:1017900090FFDFCF9091E8009E779093E800D9CF3B
:1017A0009091F200992381F09091E80090FF0CC095
:1017B0009091E80095FF03C01092F100F9CF90914D
:1017C000E8009E779093E8008F708093E9000E9474
:1017D000501084CF292F332723303105C9F060F40E
:1017E0002130310581F02230310509F041C084E714
:1017F00090E02EE233E040C021323105E1F02232A8
:10180000310531F135C082E190E022EA33E034C0A5
:1018100099278130910549F028F0029749F5E8EEC3
:10182000F2E005C0EAE2F3E002C0EAE1F3E084910D
:1018300090E09F0121C064307105D0F4660F771FDE
:10184000FB01EB5DFE4F2081318189E090E014C007
:101850006430710568F4FB01EE0FFF1FE35EFE4F7D
:1018600020813181FB01E75EFE4F808190E004C062
:1018700080E090E020E030E0FA0131832083089599
:1018800084E089BD86E089BD09B400FEFDCF80916A
:10189000D8008F7D8093D8008091E0008260809393
:1018A000E0008091E00081FDFCCF0895982F9530F5
:1018B00068F59093E900981739F07091EC00209149
:1018C000ED005091F00003C0242F762F50E021FD51
:1018D00002C09F5FECCF3091EB003E7F3093EB0076
:1018E0003091ED003D7F3093ED003091EB003160A1
:1018F0003093EB007093EC002093ED005093F000D8
:101900002091EE0027FDE5CF80E008958F70809351
:10191000E90081E008958091520487FF11C0809111
:10192000E80082FD05C0809151048111F8CF11C0FB
:101930008091E8008B770BC080915104882349F097
:101940008091E80080FFF8CF8091E8008E77809347
:10195000E80008952091E4003091E50095E640917B
:10196000EC00842F817040FF23C08091E80080FD4F
:101970001DC080915104882399F0853099F08091A1
:10198000EB0085FD11C04091E4005091E500241763
:10199000350729F3915011F09A01E1CF84E00895C1
:1019A00082E0089583E0089581E0089580E008953D
:1019B0004091E80042FFDDCF0895CF92DF92EF9291
:1019C000FF920F931F93CF93DF93EC018B017A016A
:1019D0000E94AA0C811135C0E114F10439F0F7011D
:1019E00080819181081B190BC80FD91FC12CD12CE4
:1019F0000115110529F18091E80085FD18C080913D
:101A0000E8008E778093E8000E945010E114F10402
:101A100049F0F70180819181C80ED91ED182C08220
:101A200085E00FC00E94AA0C882311F30AC0899197
:101A30008093F10001501109FFEFCF1ADF0AD8CFD0
:101A400080E0DF91CF911F910F91FF90EF90DF9099
:101A5000CF900895209158043091590426173707E4
:101A600048F06115710539F42091E8002E77209334
:101A7000E80001C0B901FC0120E06115710561F1C8
:101A8000809151048823D9F18530D9F18091E80003
:101A900083FD39C08091E80082FD2BC08091E80071
:101AA00080FFEBCF8091F20090E06115710551F05D
:101AB0008830910538F421912093F100615071092B
:101AC0000196F3CF21E0089709F020E08091E8002B
:101AD0008E778093E800D1CF2111D2CF0AC08091B8
:101AE0005104882361F0853061F08091E80083FD26
:101AF0000AC08091E80082FFF2CF80E0089582E082
:101B0000089583E0089581E008952091580430916C
:101B100059042617370748F06115710539F42091EB
:101B2000E8002E772093E80001C0B901FC0120E015
:101B30006115710579F180915104882309F43DC044
:101B4000853009F43CC08091E80083FD3AC0809163
:101B5000E80082FD2CC08091E80080FFE9CF8091F1
:101B6000F20090E06115710559F08830910540F45C
:101B700024912093F1003196615071090196F2CFC2
:101B800021E0089709F020E08091E8008E778093AB
:101B9000E800CECF2111CFCF0AC080915104882315
:101BA00061F0853061F08091E80083FD0AC080918A
:101BB000E80082FFF2CF80E0089582E0089583E09C
:101BC000089581E008951F93CF93DF93CDB7DEB7DB
:101BD000AA970FB6F894DEBF0FBECDBFE2E5F4E0E2
:101BE0008091F100819324E0EA35F207C9F70E9461
:101BF0006A0A8091E80083FF2EC18091520490917F
:101C00005304492F50E04A30510508F024C1FA012D
:101C1000E65CFF4F0C947526803821F0823809F07D
:101C20001AC108C080914E0490914F04992389F005
:101C300082600FC0809156048F70853008F00BC110
:101C40008093E9008091EB0085FB882780F9109252
:101C5000E9009091E800977F9093E8008093F1006D
:101C60001092F100D1C0282F2D7F09F0F4C08823F5
:101C700019F0823061F0EFC080915404813009F096
:101C8000EAC0933009F080E080934F042EC0809129
:101C9000540481112AC0809156048F702FEF280FB1
:101CA000243008F0D8C08093E9002091EB0020FF99
:101CB0001CC0933021F48091EB00806214C090919D
:101CC000EB0090619093EB0021E030E0A90102C0AD
:101CD000440F551F8A95E2F74093EA001092EA00FC
:101CE0008091EB0088608093EB001092E900809176
:101CF000E800877F8093E8000E948B0CACC08111C4
:101D0000AAC0109154041F778091E3008078812B42
:101D10008093E3008091E800877F8093E8000E9431
:101D20008B0C8091E80080FFFCCF8091E3008068FD
:101D30008093E300111102C082E001C083E0809330
:101D4000510489C08058823008F085C080915404C5
:101D5000909155048C3D53E0950779F583E08A8393
:101D60008AE289834FB7F894DE01139620E03EE0C3
:101D700051E2E32FF0E050935700E49120FF03C0BD
:101D8000E295EF703F5FEF708E2F90E0EA3010F039
:101D9000C79601C0C0968D939D932F5F243149F75C
:101DA0004FBF8091E800877F8093E8006AE270E08F
:101DB000CE0101960E942A0D16C0609156047091C2
:101DC0005704AE014F5F5F4F0E94EA0BBC01892BA5
:101DD00009F441C09091E800977F9093E8008981D1
:101DE0009A810E94850D8091E8008B778093E800AE
:101DF00032C0803881F58091E800877F8093E800C9
:101E000080914D048093F1008091E8008E7772CF2D
:101E1000811121C080915404909155049927029713
:101E2000D4F48091E800877F8093E8008091540487
:101E300080934D040E948B0C80914D04811106C04B
:101E40008091E30087FD02C081E001C084E08093BF
:101E500051040E94560A8091E80083FF0AC08091D5
:101E6000E800877F8093E8008091EB008062809398
:101E7000EB00AA960FB6F894DEBF0FBECDBFDF9180
:101E8000CF911F9108950E94A00F0E94A30FE0EE32
:101E9000F0E0808181608083E8EDF0E080818F77E1
:101EA000808319BCE3E6F0E080818160808310923A
:101EB000500408950E94A00F0E94A30F8091D800A3
:101EC0008F778093D8008091D80080688093D80065
:101ED0008091D8008F7D8093D80084E089BD86E012
:101EE00089BD09B400FEFDCF1092510410924D043B
:101EF00010924F0410924E0442E060E080E00E9495
:101F0000560C8091E1008E7F8093E1008091E20089
:101F100081608093E2008091E20088608093E2001B
:101F20008091E0008E7F8093E0000895E3E6F0E08A
:101F300080818E7F808381E0809350040C945A0FBF
:101F40001092E20008951092E10008951F920F92FE
:101F50000FB60F9211242F933F934F935F936F937C
:101F60007F938F939F93AF93BF93EF93FF93809152
:101F7000E10082FF0BC08091E20082FF07C08091E8
:101F8000E1008B7F8093E1000E944F108091E1007F
:101F900080FF18C08091E20080FF14C08091E200B1
:101FA0008E7F8093E2008091E20080618093E20066
:101FB0008091D80080628093D80019BC109251049F
:101FC0000E94520A8091E10084FF30C08091E200BB
:101FD00084FF2CC084E089BD86E089BD09B400FE81
:101FE000FDCF8091D8008F7D8093D8008091E10053
:101FF0008F7E8093E1008091E2008F7E8093E200EB
:102000008091E20081608093E20080914D048823FA
:1020100011F084E007C08091E30087FD02C081E0F9
:1020200001C083E0809351040E94490A8091E1003D
:1020300083FF24C08091E20083FF20C08091E100F3
:10204000877F8093E10082E08093510410924D04D9
:102050008091E1008E7F8093E1008091E2008E7F8D
:102060008093E2008091E20080618093E20042E090
:1020700060E080E00E94560C0E94550AFF91EF91AB
:10208000BF91AF919F918F917F916F915F914F9190
:102090003F912F910F900FBE0F901F9018950895AC
:1020A000CF93809151048823A1F0C091E900CF70B3
:1020B0009091EC00892F817090FD80E8C82B1092E0
:1020C000E9008091E80083FD0E94E30DCF70C0938A
:1020D000E900CF91089590935F0380935E03089584
:1020E000E0915E03F0915F03309721F00190F08161
:1020F000E02D099480E00895EF92FF920F931F93D3
:10210000CF93DF93E0915E03F0915F033097B1F1DD
:102110008C010280F381E02D099580913C0482FFBF
:102120002DC080FF04C08FEB94E00E94D105E80130
:1021300018E089EBE82E84E0F82E80913C0480FFC3
:102140000BC088811F928F93FF92EF920E946A06C4
:102150000F900F900F900F90115021961111EDCF0D
:1021600080913C0480FF0AC087EB94E0DF91CF911F
:102170001F910F91FF90EF900C94D105DF91CF91BB
:102180001F910F91FF90EF900895E0915E03F09101
:102190005F03309721F00480F581E02D09940895C4
:1021A000CF93DF9320915C0330915D0328173907AB
:1021B00009F190935D0380935C03E0915E03F091DD
:1021C0005F033097B9F0EC010680F781E02D0995A7
:1021D00080913C0482FF0EC080FF0CC0DF93CF9340
:1021E00089EA94E09F938F930E946A060F900F9064
:1021F0000F900F90DF91CF910895CF93DF932091AF
:102200005A0330915B032817390709F190935B0358
:1022100080935A03E0915E03F0915F033097B9F029
:10222000EC010084F185E02D099580913C0482FF4A
:102230000EC080FF0CC0DF93CF9389E994E09F9399
:102240008F930E946A060F900F900F900F90DF916E
:10225000CF9108950C94D5110E94CA1D0C94BF060D
:10226000BF92CF92DF92EF92FF920F931F93CF9383
:10227000DF9300D000D01F92CDB7DEB70E94470792
:1022800001E613E0F12C8F2D0E94F207B82EF80121
:10229000C080C82639F4F3940F5F1F4FF0E1FF129E
:1022A000F2CF30C080913C0481FD0E94EA11D12C14
:1022B000EE24E3948C2D8E21F9F0D982FA8291E0FC
:1022C0008B2D8E2109F490E09B830E94D31D8160A9
:1022D000782F9D838C8349815A816B818D810E94E7
:1022E000201249815A816B817C818D810E944F1D12
:1022F000F80180818E258083D394EE0CF8E0DF1204
:10230000D9CFC9CF8FEF89838A831B820E94D31DC7
:102310008160782F9D838C8349815A816B818D8167
:102320000E9420120E944E1D0E9482200E94701066
:1023300090916003891741F10E94701080936003AF
:1023400090913C0492FF0EC090FF0CC01F928F939F
:102350008AEC94E09F938F930E946A060F900F90EF
:102360000F900F90809160030F900F900F900F903F
:102370000F90DF91CF911F910F91FF90EF90DF9021
:10238000CF90BF900C94601D0F900F900F900F9006
:102390000F90DF91CF911F910F91FF90EF90DF9001
:1023A000CF90BF9008950C94F8070895CF93C62F4F
:1023B0000E94F20721E030E002C0220F331FCA95CD
:1023C000E2F790E02823392381E0232B09F480E011
:1023D000CF910895EF92FF920F931F93CF93DF93C6
:1023E00080EE94E00E94D105C0E0D0E08DE2E82EBE
:1023F00081E0F82E05ED14E08C2F0E94F2070E9478
:102400003C1DFF92EF921F928F93DF93CF931F9308
:102410000F930E946A0621968DB79EB708960FB655
:10242000F8949EBF0FBE8DBFC031D10529F7DF9153
:10243000CF911F910F91FF90EF9008950895089507
:10244000CF93DF93CDB7DEB72B970FB6F894DEBFEF
:102450000FBECDBF942F4F83252F588769877A876A
:102460008B874A855B85452B31F02F3F31F481E026
:102470009F3F19F403C081E001C080E080FD07C0E8
:102480004F81588569857A858B850E944F1DDE01B5
:10249000119686E0FD0111928A95E9F785E0FE012B
:1024A000379601900D928A95E1F749815A816B81A7
:1024B0007C818D819E810E94A5192B960FB6F89480
:1024C000DEBF0FBECDBFDF91CF910895CF93DF93D5
:1024D000882309F48FC0C82F8EE78C0F833018F53E
:1024E000C23829F0C33831F0C4E0D7E405C0C2E0F7
:1024F000D9E302C0C1E0D3E50E9470108C2309F03B
:1025000079C08D2F0E94991C0E94111D2FEF81EE22
:1025100094E0215080409040E1F700C000008D2FF2
:102520000E94B61C10C08CEF8C0F813A20F080E521
:102530008C0F8E3260F48C2F0E94AD2381115AC013
:102540008C2F0E94991CDF91CF910C94111D80E279
:102550008C0F883048F4C77081E001C0880FCA959D
:10256000EAF70E94D71CEFCF8BE58C0F833080F405
:10257000C53A29F0C63A31F083E890E005C081E819
:1025800090E002C082E890E0DF91CF910C94D010EF
:1025900088E58C0F873170F5C83A89F0C93A91F017
:1025A000CA3A99F0CB3AA1F0CC3AA9F0CD3AB1F0C1
:1025B000CE3AB9F0CF3AC1F080E090E017C082EE99
:1025C00090E014C089EE90E011C08AEE90E00EC059
:1025D00085EB90E00BC086EB90E008C083EB90E0C9
:1025E00005C084EB90E002C087EB90E0DF91CF91D3
:1025F0000C94FD10DF91CF910895CF93DF93882342
:1026000009F454C09EE7980F933008F5823829F0FA
:10261000833831F0C4E0D7E405C0C2E0D9E302C09A
:10262000C1E0D3E50E9470108C2309F43FC08D2FC8
:102630000E94991C0E94111D2FEF81EE94E0215001
:1026400080409040E1F700C000008D2F08C09CEF53
:10265000980F913A20F090E5980F9E3218F40E945E
:10266000B61C0DC090E2980F983068F4877091E026
:1026700001C0990F8A95EAF7892F0E94DD1CDF912E
:10268000CF910C94111D9BE5980F933030F480E0AE
:1026900090E0DF91CF910C94D010885A873130F4BC
:1026A00080E090E0DF91CF910C94FD10DF91CF910D
:1026B0000895882321F00E94D71C0C94111D0895C1
:1026C000882321F00E94DD1C0C94111D08950E94A6
:1026D000F71C0E94C61C0E94111D0E9428210E9406
:1026E000F51F80E090E00E94D01080E090E00C9414
:1026F000FD100E94E71C0C946713CF92DF92EF92BB
:10270000FF920F931F93CF93DF9300D000D01F92BF
:10271000CDB7DEB76C010E94621D811118C385E040
:10272000F601DE01119601900D928A95E1F7F6010E
:1027300040815181238134812115310531F05F3F82
:1027400031F481E04F3F19F403C081E001C080E023
:1027500080FDFDC2F601F280E580E2948FE0E82280
:1027600049835A83FB82722F3D832C836F2D8D8189
:102770000E940E1C8C010E940D1C0E94FD1AE12F6C
:10278000E295EF708E2F90E0FC01EC5BFF4F0C9414
:102790007526812F807F1F70882311F01295107F7E
:1027A000FF20B9F0112329F0812F0E94EA1C0E941A
:1027B000111D802F0F900F900F900F900F90DF91B1
:1027C000CF911F910F91FF90EF90DF90CF900C94DD
:1027D0006612802F0E94FD12112309F4B8C2812FC6
:1027E0000E94F01C0F900F900F900F900F90DF91B0
:1027F000CF911F910F91FF90EF90DF90CF900C94AD
:10280000111D812F807F1F70803211F01295107F73
:10281000002319F0013009F12BC0FF20A9F0EE20B0
:1028200059F1F1E0812FEF1228C00F900F900F9017
:102830000F900F90DF91CF911F910F91FF90EF902C
:10284000DF90CF900C94FA1CEE2021F021E0E216EC
:1028500009F47DC20E94FD1C4DC0FF20E9F085E017
:102860008E1508F474C20E94D41C812329F042C042
:10287000FF20F1F1E11015C0812F0F900F900F9004
:102880000F900F90DF91CF911F910F91FF90EF90DC
:10289000DF90CF900C94591394E09E1508F457C222
:1028A00029C0F601858180FF13C08F708583E4CF36
:1028B000003F09F489C108F055C180E4800F8032DF
:1028C00008F459C1FF2009F4EAC1EE2009F49AC1C5
:1028D000802F0E946612093309F0DAC1FFEF21EE62
:1028E00084E0F15020408040E1F700C000002FC29A
:1028F000E110D7C1812F59C1812F869586958370AC
:1029000019F08130B9F023C2FF2019F0C80193708B
:1029100002C080E090E00F900F900F900F900F900A
:10292000DF91CF911F910F91FF90EF90DF90CF90AB
:102930000C94D010FF2019F0C801937002C080E001
:1029400090E00F900F900F900F900F90DF91CF912C
:102950001F910F91FF90EF90DF90CF900C94FD109E
:10296000802FFF2019F00E94081F02C00E94701FD4
:102970000F900F900F900F900F90DF91CF911F91BC
:102980000F91FF90EF90DF90CF900C94F51F812F67
:10299000837009F070C0F110DAC1202F22952695BE
:1029A0002770220F220F602F6F70862F90E0A0E01B
:1029B000B0E06C017D01022E04C0CC0CDD1CEE1CCD
:1029C000FF1C0A94D2F704FF12C08FE090E0A0E051
:1029D000B0E004C0880F991FAA1FBB1F2A95D2F729
:1029E000BC01CD01609570958095909503C060E025
:1029F00070E0CB011695169513701230B1F040F5CA
:102A00006C297D298E299F29113031F10F900F906B
:102A10000F900F900F90DF91CF911F910F91FF902A
:102A2000EF90DF90CF900C94221B6C297D298E298A
:102A30009F290F900F900F900F900F90DF91CF91E3
:102A40001F910F91FF90EF90DF90CF900C943C1B63
:102A50000E94221BC701B6010F900F900F900F909C
:102A60000F90DF91CF911F910F91FF90EF90DF902A
:102A7000CF900C94081BFF2019F0812F817001C0AA
:102A80008695882309F463C1202F22952695277007
:102A9000220F220F602F6F70862F90E0A0E0B0E031
:102AA0006C017D01022E04C0CC0CDD1CEE1CFF1C51
:102AB0000A94D2F704FF12C08FE090E0A0E0B0E0EB
:102AC00004C0880F991FAA1FBB1F2A95D2F7BC010B
:102AD000CD01609570958095909503C060E070E0A1
:102AE000CB011695169513701230B1F040F56C2994
:102AF0007D298E299F29113031F10F900F900F9071
:102B00000F900F90DF91CF911F910F91FF90EF9059
:102B1000DF90CF900C94E91B6C297D298E299F2989
:102B20000F900F900F900F900F90DF91CF911F910A
:102B30000F91FF90EF90DF90CF900C94FB1B0E94C1
:102B4000E91BC701B6010F900F900F900F900F90E7
:102B5000DF91CF911F910F91FF90EF90DF90CF9079
:102B60000C94D71B023F09F45EC008F449C0033F30
:102B700009F46CC0A7CE902F9071E92E812F8F7130
:102B8000FF2051F00E94701B802FEE2019F08295DB
:102B9000807F73CE8F7071CE0E94911B802FEE20AC
:102BA00019F08295807F01C08F700F900F900F9069
:102BB0000F900F90DF91CF911F910F91FF90EF90A9
:102BC000DF90CF900C946013FF20A9F0E4E0EE15A5
:102BD00008F4BDC0812F8F710F900F900F900F9050
:102BE0000F90DF91CF911F910F91FF90EF90DF90A9
:102BF000CF900C94B61BF5E0FE1508F4A8C0EACF00
:102C0000FF2099F0812F8F710F900F900F900F90F0
:102C10000F90DF91CF911F910F91FF90EF90DF9078
:102C2000CF900C94701BFF2069F3812F8F710F9050
:102C30000F900F900F900F90DF91CF911F910F91F8
:102C4000FF90EF90DF90CF900C94911BFF2089F0C4
:102C5000812F8F710F900F900F900F900F90DF9139
:102C6000CF911F910F91FF90EF90DF90CF900C9438
:102C70005B1B0F900F900F900F900F90DF91CF91F3
:102C80001F910F91FF90EF90DF90CF900C94561B07
:102C9000033509F423CE073409F059C01FCEEE20C6
:102CA00021F2802F0F900F900F900F900F90DF91D7
:102CB000CF911F910F91FF90EF90DF90CF900C94E8
:102CC000FD12412F4F70602FC6010E947E1E0F9093
:102CD0000F900F900F900F90DF91CF911F910F9158
:102CE000FF90EF90DF90CF900C94581A01112FC0F5
:102CF000FF2069F10E9479132FEF80E792E02150C5
:102D000080409040E1F700C000000F900F900F90BE
:102D10000F900F90DF91CF911F910F91FF90EF9047
:102D2000DF90CF900C94201E412F4F70602FC60172
:102D30000F900F900F900F900F90DF91CF911F91F8
:102D40000F91FF90EF90DF90CF900C94811E0F9029
:102D50000F900F900F900F90DF91CF911F910F91D7
:102D6000FF90EF90DF90CF9008951F93CF93DF9364
:102D700000D000D01F92CDB7DEB7942F4983252F06
:102D80005A836B837C838D834C815D81452B31F02D
:102D90002F3F31F481E09F3F19F403C081E001C06F
:102DA00080E0182F117080FD31C049815A816B81FC
:102DB0007C818D810E940E1C292F22952F702C3032
:102DC00030F42A30A0F42250223030F022C02C30CF
:102DD000C9F02F30B9F01DC0853A28F48430C0F412
:102DE000823028F415C090E2980F983088F0883E21
:102DF00030F4803E68F48450813A58F409C0803F32
:102E000041F406C093FB112710F903C010E001C084
:102E100011E0812F0F900F900F900F900F90DF9186
:102E2000CF911F910895CF93DF9300D000D01F92D0
:102E3000CDB7DEB70F900F900F900F900F90DF91EE
:102E4000CF910895CF93DF9300D000D000D0CDB7BD
:102E5000DEB726960FB6F894DEBF0FBECDBFDF916A
:102E6000CF910895CF93DF93C09171038091720346
:102E7000C817A1F0D0E0CE0166E070E00E945026B5
:102E8000FC01ED58FC4F4081518162817381848146
:102E900095810E9422172196C770E8CFDF91CF91CC
:102EA00008954091A3035091A4036091A5037091EC
:102EB000A6038091A7039091A8030C9422171F9357
:102EC000CF93DF938091A80382958F7009F05CC047
:102ED0008091A503882309F457C0209171031091B4
:102EE0007203C091A303D091A403A091A603B09153
:102EF000A70381E0CF3F09F080E0482F211709F4B4
:102F000043C0109721F0DF3F21F080E003C081E053
:102F100001C0842F30E080FD33C0C90166E070E05D
:102F20000E945026FC01ED58FC4F81818D1328C072
:102F300080818C1325C08281811122C0838194817C
:102F40008A1B9B0B883C9105D8F48091A8038F7055
:102F500080618093A803C90166E070E00E9450265A
:102F6000FC01E858FC4F90819F709061908383EA48
:102F700093E00E947D13DF91CF911F910C94321743
:102F80002F5F3F4F2770BACFDF91CF911F910895E8
:102F90009F92AF92BF92CF92DF92EF92FF920F93E8
:102FA0001F93CF93DF93CDB7DEB761970FB6F89439
:102FB000DEBF0FBECDBF8C0185E0F801DE011D969E
:102FC00001900D928A95E1F7F80140812181F2800C
:102FD000C380D4809091A3033091A4036091A60391
:102FE0007091A7036115710531F03F3F31F481E025
:102FF0009F3F19F403C081E001C080E0F82FF17019
:103000009F2E80FD59C183EAA82E83E0B82EE09060
:10301000A503F601E61BF70BEE2009F4EDC0809145
:10302000A803582F507FE83CF10508F0A7C05111C4
:1030300056C0231313C0491311C0EF2CF1100EC05A
:103040008F7080618093A8030E945117C5010E9470
:103050007D138091A803F801858364C1C114D10454
:1030600031F02F3F31F481E04F3F19F403C081E08C
:1030700001C080E080FD03C081E08F2502C080E0B8
:1030800090E0F82FF170EF2E80FF1FC0E0917103E8
:1030900030917203E31709F421C1F0E0CF0166E03B
:1030A00070E00E945026DC01AD58BC4F11968C9107
:1030B0001197281307C08C91481304C012968C9165
:1030C000F81203C03196E770E5CFEF2CFF2009F42A
:1030D00029C18091A80381608093A80364C0231351
:1030E00006C0491304C0F11002C0F801A9C04D8701
:1030F0002E87FF867C2DD98AC88A522F6F2D898909
:103100000E94B5168823A1F1FF2091F12091A80318
:10311000822F82958F7090E0029774F08091A303C4
:103120009091A40398878F831986DB86CA862C87A3
:10313000CE0107960E947D1386E0F801A3EAB3E072
:1031400001900D928A95E1F70E945F170E94511736
:1031500012C0231751F14D872E87FF867C2DD98A07
:10316000C88A522F6F2D89890E94B51681112CC0F3
:10317000C8010E947D13EE24E394D4C05111E9CF1D
:103180007C2DD98AC88A522F6F2D89890E941317E6
:1031900083EA93E00E947D1386E0F50111928A95FF
:1031A000E9F70E945117E12CBDC04913D4CFF110AB
:1031B000D2CFF8018583C8010E947D1386E0F50116
:1031C00011928A95E9F7AEC0FF2091F22091A803F1
:1031D000822F82958F7090E002970CF4ADCF809192
:1031E000A3039091A4039A8389831B82DD82CC82FE
:1031F0002E83CE0101969ECFE83CF10508F04CC02D
:10320000EF2CFF2009F4B4CF231330C049132EC094
:103210002091A80320FD21C0822F82958F70482F16
:1032200050E041155105C9F0F80125834F30510593
:1032300041F08F5F982F9295907F822F8F70892B0E
:103240008583C8010E947D1386E0F801A3EAB3E0FC
:1032500001900D928A95E1F72CC086E0F801A3EA6F
:10326000B3E001900D928A95E1F75CC04D872E87FF
:10327000FF867C2DD98AC88A522F6F2D89890E949A
:10328000B516811159CF8091A80381608093A8035E
:10329000C8010E947D1346C07C2DD98AC88A522F4E
:1032A0006F2D89890E94131786E0F50111928A9586
:1032B000E9F70E94511736C0FF2009F459CF4D8716
:1032C0002E87FF867C2DD98AC88A522F6F2D898937
:1032D0000E94B516882309F44BCF2ECF7C2DD98AB6
:1032E000C88A522F6F2D89890E940E1C292F229582
:1032F0002F70223028F49F7039F0811105C00BC067
:10330000243028F49F7049F4805E883020F0C80192
:103310000E947D139E2CE92C05C0F8019581907FB9
:1033200099F7F9CF8E2D61960FB6F894DEBF0FBED8
:10333000CDBFDF91CF911F910F91FF90EF90DF9064
:10334000CF90BF90AF909F900895CF93DF93CDB76C
:10335000DEB72C970FB6F894DEBF0FBECDBF4F83FC
:10336000588769877A878B879C87CE0107960E944A
:10337000C8178823D1F09F8188852A853B85232B18
:1033800031F08F3F31F481E09F3F19F403C081E0B9
:1033900001C080E080FD6FC04F81588569857A85C6
:1033A0008B859C850E94221766C086E0FE013796B9
:1033B000DE01119601900D928A95E1F7FF81E88573
:1033C0006A857B856115710531F0EF3F31F481E04D
:1033D000FF3F19F403C081E001C080E080FD4BC0D5
:1033E0008091720390E09C012F5F3F4F277033273D
:1033F0004091710350E02417350709F443C0F98365
:10340000EA837D836C8366E070E00E945026DC01D5
:10341000AD58BC4F96E0FE01319601900D929A9501
:10342000E1F7209372030E94321725C090E066E016
:1034300070E00E9450268D589C4F0E94C817882328
:1034400071F18091710390E066E070E00E94502677
:10345000FC01ED58FC4F4081518162817381848170
:1034600095810E9422178091710390E001968770E8
:10347000992780937103809171039091720389134E
:10348000D5CF0DC00E947913109272031092710370
:10349000E3EAF3E086E0DF011D928A95E9F72C96D6
:1034A0000FB6F894DEBF0FBECDBFDF91CF91089568
:1034B000DF92EF92FF920F931F93CF93DF93FC0164
:1034C000892B09F488C0E12CF12CDD24D394EF0181
:1034D00021968491853709F460C058F4843708F048
:1034E0004EC0843008F068C08130D1F0823071F174
:1034F00072C0883709F45BC050F4863709F453C0B2
:10350000873709F068C08E2D0E94E41C52C09CE7EA
:10351000980F903708F05FC08F770E94FD124EC061
:103520008F010E5F1F4FFE01849190E2980F98303B
:1035300050F48770FD2D01C0FF0F8A95EAF78F2F99
:103540000E94EA1C15C00E94661214C08F010E5F13
:103550001F4FFE01849190E2980F983068F48770B5
:10356000FD2D01C0FF0F8A95EAF78F2F0E94F01CF6
:103570000E94111DE80122C00E94FD12FBCFCF0165
:103580000296FE01C491CC2361F0EFE9FFE0319790
:10359000F1F700C00000C150F6CFCF010296FE0146
:1035A000F490EC010BC00E94D41CE82E07C00E94CE
:1035B000E71C0E94111D02C00E9466128F2D8823F5
:1035C00041F0EFE9FFE03197F1F700C000008150D2
:1035D000F6CFFE017CCFDF91CF911F910F91FF902D
:1035E000EF90DF9008956093290470932A048093EC
:1035F0002B0490932C040C945F1D089560932D046C
:1036000070932E0480932F04909330040C945E1DCD
:103610000F931F9300912D0410912E0420912F04DD
:1036200030913004602B712B822B932B60932D04EF
:1036300070932E0480932F04909330041F910F9168
:103640000C945E1D0F931F9300912D0410912E0476
:1036500020912F043091300460237123822393231F
:1036600060932D0470932E0480932F049093300464
:103670001F910F910C945E1D0F931F9300912D04C9
:1036800010912E0420912F0430913004602771276F
:103690008227932760932D0470932E0480932F0428
:1036A000909330041F910F910C945E1D60E070E0C8
:1036B000CB010C94F31A0F931F9341E050E060E0AC
:1036C00070E08A019B0104C0000F111F221F331FED
:1036D0008A95D2F7C901B8011F910F910C94F31A82
:1036E0000F931F9341E050E060E070E004C0440F8E
:1036F000551F661F771F8A95D2F7809129049091F4
:103700002A04A0912B04B0912C048A019B01082B60
:10371000192B2A2B3B2BC901B8011F910F910C9437
:10372000F31A0F931F9341E050E060E070E004C093
:10373000440F551F661F771F8A95D2F74095509505
:10374000609570958091290490912A04A0912B0492
:10375000B0912C048A019B01082319232A233B23BF
:10376000C901B8011F910F910C94F31A0F931F9385
:1037700041E050E060E070E004C0440F551F661F58
:10378000771F8A95D2F78091290490912A04A091FD
:103790002B04B0912C048A019B01082719272A27A2
:1037A0003B27C901B8011F910F910C94F31A0F9395
:1037B0001F930091290410912A0420912B04309129
:1037C0002C04602B712B822B932B1F910F910C9447
:1037D000F31A0F931F930091290410912A0420914A
:1037E0002B0430912C0460237123822393231F9197
:1037F0000F910C94F31A0F931F93009129041091C9
:103800002A0420912B0430912C04602771278227F1
:1038100093271F910F910C94F31A08958F929F9202
:10382000AF92BF92DF92EF92FF920F931F93CF93CD
:10383000DF9300D000D01F92CDB7DEB76B837C83BF
:103840008D838A018C819D81892B31F01F3F31F45A
:1038500081E04F3F19F403C081E001C080E080FFA8
:1038600003C080E090E054C08B81882309F43DC000
:103870008090290490902A04A0902B04B0902C04EE
:1038800080912D0490912E04A0912F04B0913004CA
:10389000882A992AAA2ABB2A2FE1E22EF12CD501E7
:1038A000C4010E2C04C0B695A795979587950A94E8
:1038B000D2F780FD06C081E0E81AF10880F7D12C2C
:1038C00007C0DE2CB8018E2D0E94511E019799F37E
:1038D000E12FF0E093E0EE0FFF1F9A95E1F7E75537
:1038E000FC4FE00FF11DD0820CC0E12FF0E083E02F
:1038F000EE0FFF1F8A95E1F7E755FC4FE00FF11D32
:10390000D08009831A8369817A818D2D0E94511E8E
:103910000F900F900F900F900F90DF91CF911F910C
:103920000F91FF90EF90DF90BF90AF909F908F909E
:1039300008952091110130911201F90132969FEF03
:1039400040E05191851789F09F3F19F4511101C052
:10395000942F4F5F4630A9F79F3F39F0F901E90FE7
:10396000F11D97FDFA95828308950895E091110164
:10397000F09112019F012A5F3F4F9281891301C08C
:1039800012823196E217F307C1F7089581E090E0C3
:10399000E0911101F0911201E80FF91F10820196D8
:1039A00088309105A9F7089580913B04089590917E
:1039B0003B04892B80933B040895809590913B04B0
:1039C000892380933B04089580933B0408951092CB
:1039D0003B04089590913A04892B80933A0408950A
:1039E000809590913A04892380933A040895109227
:1039F0003A04089580933104089510923104089593
:103A00008091110190911201FC0131969C01285F77
:103A10003F4F80E0919191118F5FE217F307D1F74B
:103A20000895E0911101F091120180913B0480838F
:103A3000E0911101F0911201908180913A04892B5B
:103A4000808380913104882361F0E0911101F0912D
:103A500012019081892B80830E94001D8111109298
:103A6000310480911101909112010C947C1090937B
:103A700039018093380108958295982F9373292FE7
:103A8000220F220F982F9C7C96959695922B892F2A
:103A90008575880F9A7A9695892B08950895CF9306
:103AA000DF9300D000D01F92CDB7DEB70F900F90FC
:103AB0000F900F900F90DF91CF9108950895089582
:103AC0000C94D31180E0089580915104843021F149
:103AD00010923D0420E488E190E00FB6F894A89598
:103AE000809360000FBE2093600083B7817F846065
:103AF00083BF83B7816083BF7894889583B78E7FB7
:103B000083BF0FB6F894A895809160008861809378
:103B10006000109260000FBE0895CF930E941E12A5
:103B20000E9447070E941F12C0E08C2F0E94F207DC
:103B3000811104C0CF5FC031C1F701C081E0CF91D6
:103B400008951F920F920FB60F9211248F939F9397
:103B5000AF93BF9380913D04811113C080913E04C7
:103B600090913F04A0914004B09141044196A11D61
:103B7000B11D80933E0490933F04A0934004B09302
:103B80004104BF91AF919F918F910F900FBE0F9005
:103B90001F90189582E084BD93E095BD9AEF97BD84
:103BA00080936E0008952FB7F89480913E04909111
:103BB0003F04A0914004B09141042FBF08952FB756
:103BC000F89460913E0470913F048091400490917C
:103BD00041042FBF08959C014FB7F89480913E0493
:103BE00090913F04A0914004B09141044FBF821BCB
:103BF000930B089578941F920F920FB60F92112491
:103C00008F939F93AF93BF9380913E0490913F0415
:103C1000A0914004B09141040196A11DB11D809373
:103C20003E0490933F04A0934004B0934104BF919D
:103C3000AF919F918F910F900FBE0F901F9018958D
:103C40000E94430FF89487E797E7909301088093C9
:103C5000000887E090EBDC0180935A0490935B04AA
:103C6000A0935C04B0935D049CE088E10FB6F894E7
:103C7000A895809360000FBE90936000FFCFE92F5E
:103C8000F0E093E0EE0FFF1F9A95E1F7E80FF11DCA
:103C9000E855FE4F8491982F92959F708F70977082
:103CA0000895CF93C82FCB010E943F1E292F30E0EB
:103CB00054E0220F331F5A95E1F7282B20383105A5
:103CC0001CF080E090E018C0EC2FF0E023E0EE0F55
:103CD000FF1F2A95E1F79770E90FF11D34E0EE0F11
:103CE000FF1F3A95E1F78F70E80FF11DEE0FFF1FF0
:103CF000E855FF4F85919491CF91089580E090E031
:103D0000089508958091440480FF0CC080911601AD
:103D100090E065E070E00E94502695958795959516
:103D200087952EC081FF0AC08091160190E065E062
:103D300070E00E9450269595879522C082FF08C0AA
:103D40008091160190E065E070E00E94502618C056
:103D5000209145042223D9F030911501231780F7D3
:103D60008091160190E065E070E00E945026622F7D
:103D700070E00E945026632F70E00E946126CB0104
:103D80008038910538F4009739F481E005C085E06A
:103D900090E008958FE7089508958091440480FF8E
:103DA00008C06091140170E07595679575956795E9
:103DB00023C081FF06C06091140170E0759567957E
:103DC0001BC082FF04C06091140170E012C06091BA
:103DD00045046623A9F0209113016217A0F7809192
:103DE000140170E090E00E945026622F70E00E9463
:103DF00061266038710540F46115710519F406C03B
:103E000061E070E0862F08958FE7089581E00895BE
:103E1000803F21F40E94821E819504C0813F29F4D5
:103E20000E94821E809348040895823F21F40E94DC
:103E3000821E819504C0833F29F40E94821E8093D4
:103E400047040895893F19F40E94CD1E05C08A3F9A
:103E500031F40E94CD1E81958093490408958B3FD3
:103E600021F40E94CD1E819504C08C3F29F40E944C
:103E7000CD1E80934A040895843F21F48091460426
:103E8000816017C0853F21F480914604826011C093
:103E9000863F21F48091460484600BC0873F21F463
:103EA00080914604886005C0883F31F480914604C3
:103EB00080618093460408958D3F21F480914404ED
:103EC00081600BC08E3F21F480914404826005C064
:103ED0008F3F29F4809144048460809344040895C2
:103EE000803F39F48091480487FF6CC010924804E9
:103EF00069C0813F29F4809148041816BCF362C060
:103F000090914704823F29F497FF5CC010924704C8
:103F100059C0833F19F41916CCF354C0893F41F4BA
:103F20008091490418160CF04DC0109249044AC003
:103F30008A3F29F48091490487FF44C0F6CF8B3F24
:103F400039F480914A0487FF3DC010924A043AC078
:103F50008C3F29F480914A041816BCF333C0843F87
:103F600021F4809146048E7F17C0853F21F4809113
:103F700046048D7F11C0863F21F4809146048B7FDB
:103F80000BC0873F21F480914604877F05C0883F9E
:103F900031F4809146048F7E8093460413C08D3F98
:103FA00021F4809144048E7F0BC08E3F21F48091D8
:103FB00044048D7F05C08F3F29F4809144048B7F9A
:103FC000809344048091470481110EC0809148047D
:103FD00081110AC080914904811106C080914A0470
:103FE000811102C010924504089580913C0483FF22
:103FF0007EC084E195E00E94D105809146041F9225
:104000008F938FE095E09F938F930E946A068DE0D7
:1040100095E00E94D10580914704282F082E000CBE
:10402000330B3F938F938AE095E09F938F930E9489
:104030006A0688E095E00E94D10580914804282F07
:10404000082E000C330B3F938F9385E095E09F93F0
:104050008F930E946A0683E095E00E94D1058091CB
:104060004904282F082E000C330B3F938F9380E0D8
:1040700095E09F938F930E946A068EEF94E00E94D2
:10408000D10580914A04282F082E000C330B3F9352
:104090008F938BEF94E09F938F930E946A0688EF33
:1040A00094E00E94D105809145041F928F9385EF83
:1040B00094E09F938F930E946A0683EF94E00E949E
:1040C000D105809144041F928F9380EF94E09F93D9
:1040D0008F930E946A068DEE94E00E94D1058DB701
:1040E0009EB74C960FB6F8949EBF0FBE8DBF86E468
:1040F00094E00E94C5100E94D31D909343048093C6
:10410000420408951F93CF93DF93809142049091CE
:1041100043040E94EB1DFC0120914504222321F061
:104120008091170190E007C08091180190E06AE04B
:1041300070E00E945026E817F90708F485C08091C6
:104140004704C0914804D091490410914A04811158
:1041500007C0C11175C0D11173C0111171C074C0F5
:104160002F3F19F02F5F20934504181624F40E9466
:10417000821E809347048091470487FF05C00E94F8
:10418000821E8195809347041C1624F40E94821E8F
:10419000809348048091480487FF05C00E94821ED6
:1041A00081958093480460914704662331F1C09162
:1041B0004804CC2311F1062E000C770B880B990BC9
:1041C0000E944F2523E333E343E35FE30E94B325DB
:1041D0000E941725609347046C2FCC0F770B880B38
:1041E000990B0E944F2523E333E343E35FE30E94EF
:1041F000B3250E941725609348041D1624F40E94DD
:10420000CD1E809349048091490487FF05C00E9418
:10421000CD1E819580934904111624F40E94CD1E71
:1042200080934A0480914A0487FF05C00E94CD1EF6
:10423000819580934A04DF91CF911F910C94F51FD3
:104240002F3F09F08FCFA0CFDF91CF911F9108951D
:10425000E6E4F4E085E0DF011D928A95E9F710922B
:10426000450410924404089587E397E00E94D10525
:104270001F9281E08F931F9285E08F9389EE96E0E5
:104280009F938F930E946A060F900F900F900F904C
:104290000F900F9008958330E9F128F4813061F098
:1042A000823009F10895853009F462C008F449C0EC
:1042B000863009F474C0089580911801262F30E0EB
:1042C000280F311D2F3F310524F4680F609318012A
:1042D00003C08FEF80931801809118011F928F9374
:1042E00082E296E072C080911701262F30E0280FFD
:1042F000311D2F3F310524F4680F6093170103C06F
:104300008FEF80931701809117011F928F9380E1A7
:1043100096E05BC080911601262F30E0280F311DFA
:104320002F3F310524F4680F6093160103C08FEF0F
:1043300080931601809116011F928F938DEF95E067
:1043400044C080911501262F30E0280F311D2F3FEA
:10435000310524F4680F6093150103C08FEF80933B
:104360001501809115011F928F9388EE95E02DC065
:1043700080911401262F30E0280F311D2F3F310589
:1043800024F4680F6093140103C08FEF809314012D
:10439000809114011F928F938FEC95E016C080914D
:1043A0001301262F30E0280F311D2F3F310524F453
:1043B000680F6093130103C08FEF80931301809106
:1043C00013011F928F9384EB95E09F938F930E942C
:1043D0006A060F900F900F900F900895833081F12F
:1043E00028F4813059F08230D1F00895853009F4F5
:1043F00049C0B8F1863009F456C00895809118017B
:10440000681720F4861B8093180102C010921801CF
:10441000809118011F928F9385EA95E054C0809196
:104420001701681720F4861B8093170102C01092B1
:104430001701809117011F928F9383E995E043C084
:1044400080911601681720F4861B8093160102C024
:1044500010921601809116011F928F9380E895E0CB
:1044600032C080911501681720F4861B80931501D6
:1044700002C010921501809115011F928F938BE657
:1044800095E021C080911401681720F4861B809369
:10449000140102C010921401809114011F928F9395
:1044A00082E595E010C080911301681720F4861B07
:1044B0008093130102C010921301809113011F9287
:1044C0008F9387E395E09F938F930E946A060F90E6
:1044D0000F900F900F900895CF93C82F1F928F9336
:1044E0008CE398E09F938F930E946A0681E090E0AE
:1044F000A0E0B0E0BC01CD0104C0660F771F881FAB
:10450000991FCA95D2F70E94FE1A0F900F900F9034
:104510000F90CF910C947913CF93873288F58E3119
:1045200008F00BC18E3009F487C0D8F4873009F445
:1045300060C08B3009F44FC0863009F002C1809111
:104540003C04817F8E7F80933C0481E498E00E944C
:10455000D10582EF9AE00E94D10581E080934C045E
:1045600046C0863109F4B0C020F4803109F47AC025
:10457000E8C0893109F491C08B3109F449C0E1C028
:10458000883349F150F4893209F4D5C0853309F4F0
:10459000D2C0873209F0D5C0CEC0833409F4CBC075
:1045A00028F48A3308F4CDC08953C8C0883409F090
:1045B000C8C00E94791381EE9AE00E94D1052FEFC6
:1045C00083ED90E3215080409040E1F700C000006F
:1045D0000E94201E0CC088E698E041C088EC9AE05A
:1045E0000E94D10580913C04816080933C04C1E02D
:1045F000ADC080913C04C82FC17080FFEFCF84ED27
:104600009AE00E94D10580913C04817F8E7F3FC05B
:1046100090913C0491FBCC27C0F981E0C827892FF9
:10462000C0FB81F980933C04CC2319F08BEB9AE01A
:1046300029C08DEA9AE013C090913C0492FBCC27EC
:10464000C0F981E0C827892FC0FB82F980933C0420
:10465000CC2319F08EE99AE015C08EE89AE00E940A
:10466000D105C5CF90913C0493FBCC27C0F981E0E4
:10467000C827892FC0FB83F980933C04CC2351F0D9
:1046800082E89AE00E94D10580913C048160809389
:104690003C045CC085E79AE0E2CF86E69AE00E949F
:1046A000D10586E39AE00E94D10580EF99E00E944F
:1046B000D10588EC99E00E94D10582E999E00E9439
:1046C000D10586E699E0CBCF88E599E00E94D10537
:1046D0000E9470101F928F938EE399E09F938F93A7
:1046E0000E946A06809110011F928F9387E299E0E1
:1046F0009F938F930E946A06809159031F928F9314
:1047000084E199E09F938F930E946A060E94DF1DC7
:104710009F938F937F936F938DEF98E09F938F93E9
:104720000E946A068DB79EB742960FB6F8949EBF58
:104730000FBE8DBF5CCF80E001C08D510E946C2206
:1047400056CF8BEF98E00E94D105C0E08C2FCF911F
:10475000089580E008950C94A9230F931F93CF939D
:10476000C82F80914C048130B1F020F0823009F4E0
:104770005BC052C160E070E08CE090E00E94D61116
:10478000892BC9F4E0911101F091120180818434E8
:1047900009F044C110C060E070E08CE090E00E943D
:1047A000D6118C01892B39F4E0911101F09112019D
:1047B0008081843461F48C2F0E94AB23811104C06A
:1047C0008C2F0E948C222EC081E090E02BC08C2F79
:1047D0000E94A923811124C1C431E1F070F4CB30CF
:1047E00081F0C031D1F40E94342184E398E00E942A
:1047F000D10582E080934C0413C1C93259F0C8330B
:1048000061F481E498E00E94D10588E398E00E9479
:10481000D10506C110924C0404C082E398E00E94C6
:10482000D105802F8170FFC0C43228F5CE3108F049
:10483000C1C0CB30A1F1D0F4C73009F0D3C08EE1B4
:104840008093180182E3809317018AE08093160118
:1048500084E18093150188E08093140188E28093BD
:10486000130188ED96E00E94D105BFC0C33149F124
:10487000C431C1F0B7C0CB3409F4A9C028F4C9329F
:1048800089F0C83361F0AEC0C13509F49EC0C235AD
:1048900009F499C0CE3409F0A5C06AE09EC00E9418
:1048A0003421A3C080914B04882319F010924B044B
:1048B0009CC085EE96E00E94D10581E080934C0477
:1048C000B2C08FEB96E00E94D1058DEA96E00E947F
:1048D000D105809118011F928F938AEA96E09F93E9
:1048E0008F930E946A0688EA96E00E94D10586E9C5
:1048F00096E00E94D105809117011F928F9383E962
:1049000096E09F938F930E946A0681E996E00E9449
:10491000D10582E896E00E94D105809116011F9290
:104920008F938FE796E09F938F930E946A068DE79F
:1049300096E00E94D1058CE696E00E94D105809118
:1049400015011F928F9389E696E09F938F930E94A3
:104950006A0687E696E00E94D10582E596E00E940D
:10496000D105809114011F928F938FE496E09F935D
:104970008F930E946A068DE496E00E94D10586E33B
:1049800096E00E94D105809113011F928F9383E3DB
:1049900096E09F938F930E946A0681E396E00E94BF
:1049A000D1058DB79EB748960FB6F8949EBF0FBE3F
:1049B0008DBF1BC0CE51EC2FF0E0E25DFE4F808139
:1049C00080934B0412C061E003C061E006C06AE05E
:1049D00080914B040E944B2108C080914B040E949F
:1049E000EE2103C086ED96E013C080914B0488232E
:1049F00069F01F928F9380ED96E09F938F930E94B2
:104A00006A060F900F900F900F9004C08DEC96E007
:104A10000E94D10581E007C010924C0480E003C0E1
:104A200001E010E0FECECF911F910F9108950E94FA
:104A30001E256894B1110C94AD2508950E9492250D
:104A400088F09F5798F0B92F9927B751B0F0E1F04F
:104A5000660F771F881F991F1AF0BA95C9F714C0FF
:104A6000B13091F00E94AC25B1E008950C94AC25D2
:104A7000672F782F8827B85F39F0B93FCCF3869538
:104A800077956795B395D9F73EF490958095709595
:104A900061957F4F8F4F9F4F0895E89409C097FB12
:104AA0003EF490958095709561957F4F8F4F9F4F05
:104AB0009923A9F0F92F96E9BB279395F695879549
:104AC00077956795B795F111F8CFFAF4BB0F11F40C
:104AD00060FF1BC06F5F7F4F8F4F9F4F16C08823B3
:104AE00011F096E911C0772321F09EE8872F762FE9
:104AF00005C0662371F096E8862F70E060E02AF02A
:104B00009A95660F771F881FDAF7880F9695879515
:104B100097F9089557FD9058440F551F59F05F3F7E
:104B200071F04795880F97FB991F61F09F3F79F0CF
:104B300087950895121613061406551FF2CF469551
:104B4000F1DF08C0161617061806991FF1CF8695D3
:104B50007105610508940895E894BB2766277727B7
:104B6000CB0197F908950E94C5250C943F260E9419
:104B7000312638F00E94382620F0952311F00C944D
:104B800028260C942E260C94AD250E948A2578F3B5
:104B90009923C9F35523B9F3950F50E0551FAA2760
:104BA000EE27FF27BB2700240894679520F4E20F27
:104BB000F31FB41F0A1E220F331F441FAA1F66953E
:104BC000A9F7779530F4F30FB41F0A1E121E08F4EC
:104BD0006395330F441FAA1F221F769599F7879577
:104BE00020F4B40F0A1E121E631F440FAA1F221FB7
:104BF000331F8695A9F7862F712D602D11249F579D
:104C000050409AF0F1F088234AF0EE0FFF1FBB1FCF
:104C1000661F771F881F91505040A9F79E3F51058E
:104C200080F00C9428260C94AD255F3FE4F3983E69
:104C3000D4F3869577956795B795F795E7959F5F38
:104C4000C1F7FE2B880F911D9695879597F90895CA
:104C500097F99F6780E870E060E008959FEF80EC2F
:104C6000089500240A9416161706180609060895D2
:104C700000240A9412161306140605060895092E38
:104C80000394000C11F4882352F0BB0F40F4BF2BA7
:104C900011F460FF04C06F5F7F4F8F4F9F4F0895E7
:104CA0000024552704C0080E591F880F991F00972C
:104CB00029F076956795B8F37105B9F7802D952F92
:104CC000089597FB072E16F4009407D077FD09D0BE
:104CD0000E947B2607FC05D03EF4909581959F4F5E
:104CE0000895709561957F4F0895EE0FFF1F059011
:104CF000F491E02D0994AA1BBB1B51E107C0AA1F28
:104D0000BB1FA617B70710F0A61BB70B881F991F6C
:104D10005A95A9F780959095BC01CD010895F89416
:024D2000FFCFC3
:104D22000550020000FF84081409F108BB08870837
:104D32000132042808140A321E404D362259040C4E
:104D420004D603B4034003590372038B0300010228
:084D520003040506070809002F
:00000001FF
